:03000000020B08E8
:03000300022003D5
:03000B0002200BC5
:08001300308A030220130145AD
:03001B0002201BA5
:0300230002202395
:03002B0002202B85
:10003000A188A180C183C1E5C1F2A1DEC104A19064
:10004000C1C30202E9C0D0C0E0C2D3C2D4B180D1E2
:10005000C3B40D020193B42002212EB43F04313306
:10006000014DB45111C082C083901457D1F2D08396
:10007000D082C2AA212EB448043152014DB452029A
:10008000219BB453024131B441024167014D743D9B
:10009000B18822E8C0E0D1DC7453B1887450B188D3
:1000A000118EA881C0F0D18318D1DC120AE8118E1C
:1000B000E6D18318D1DC120AEE118EE6A2E7E43312
:1000C000D18DD1DC120AF9118EE583D183E582D17D
:1000D00083E43143A88118E6D18374013143E9D127
:1000E0008374023143EAD18374033143EBD18374C7
:1000F000043143ECD18374053143EDD1837406316F
:1001000043EED18374073143EFD183B1A1D1DC74C5
:1001100050B188120AEE118EC3E5819404F8C082B2
:10012000C083120BA5D083D082D0F0D0E0F8D0E00D
:10013000D0D032C082C083B1A1901CD8D1F2D0837C
:10014000D08222C0E0D1DC7452B188D0E0D18D11D0
:100150008E22C000C001C0F0C082C083901422D1A2
:10016000F2D083D082E4D183743AB188D1DCE8D173
:1001700083D1DCE9D1837802790E2185E8D18374BB
:100180003AB1887910D1DCE6D18308D9F8B1A1B8A9
:1001900080EAB1A1D0F0D001D00022C0F0D1DC744F
:1001A00042B188118EE5F0D183D1DC7450B18874EE
:1001B00053B1887457B188118EE8C0E0A88118182F
:1001C00018E6D183D1DCC082C08390100EA8A8515C
:1001D00027901011A8B85127901014A88951279082
:1001E0001019A888512790101EA898512790102305
:1001F000A88751277454B1887430B188118EE58C6A
:10020000D183E58AD183D1DC7454B1887431B1884B
:10021000118EE58DD183E58BD183B1A1D083D082BE
:10022000D0E0F8D0F0014DD1F2118EE8D183D1DCCD
:1002300022C0F0E8C0E0E581C39404F8C082C08326
:10024000901400D1F2120BA5E581C39406F8A683A1
:1002500018A682901411D1F208120BA5D083D08277
:10026000D0E0F8D0F0014DE8C0E0C0F0A881181847
:10027000C082C083901447D1F2B1DE400EF6B1A126
:10028000D083D082D0F0D0E0F8014D9008ABD1F20D
:10029000D083D082D0F0D0E0F8014DC082C08390EE
:1002A000128DD1F2B180B41B0A9012D6D1F2D08354
:1002B000D08222B43AEEB1DE40EFF8B1DE40EAF58A
:1002C00083B1DE40E4F582B1DE40DEB4010A901273
:1002D000F1D1F2D083D082220841E1B1DE40CAF0F0
:1002E000A3D8F8B1DE40C241A44387807589117557
:1002F0009850438852E57BA97AAA79AB7863015577
:100300006302CC63031DB50108B50205B503028085
:1003100048C28E758D00758B0020B0FD20B0F22094
:10032000B0EF20B0EC20B0E930B0FDD28E20B0FDAF
:1003300030B0FD20B0FD30B0FDC28EE58B33E58DD1
:1003400033F404F5F0F57B6455F57AE5F064CCF50B
:1003500079E5F0641DF578E5F0F58D758921D28E8B
:1003600022C082C08390153BD1F290148CE493603C
:1003700029A3D1DCB1887804D1DCD8FCE493F5F072
:10038000A3E493A3A3A3C082C083F58285F083E492
:10039000D1F2B1A1D083D08280D4901566D1F2D0B1
:1003A00083D08222C082C083900812D1F2B180D162
:1003B000C3B41B0A9008ABD1F2D083D08222B43FE1
:1003C000239016B8D1F290083FD1F2B180B41B054A
:1003D000D083D08222901B92D1F2901CD8D1F2D03F
:1003E00083D08222B45307901336D1F28133901315
:1003F0000AD1F290084FD1F2D083D082D1E5C082E9
:10040000C0839007E8D1F2D083D082D10450069007
:1004100008ABD1F222740DB188C082C0839013174B
:10042000D1F2D083D0827400C0E07400C0E0C082FA
:10043000C0832290084FD1F2D083D082C082C08383
:10044000D1E59007E8D1F2D083D082D104C082C038
:1004500083500C9008ABD1F2B1A1D083D08222C2DC
:100460008A30B30A90134ED1F2D083D08222900802
:100470006CD1F2B180D1C3B41B0A9008ABD1F2D0D9
:1004800083D08222B44C0575B800800375B80490FF
:1004900013C4D1F2D083D0827581387400C0E07467
:1004A00000C0E0E4C3780079017A007B007C007D25
:1004B000007E007F00C28AD2B375A884737A10B11F
:1004C000A17820D1E5743AB1887420B188E493F61C
:1004D000D1837420B188A308B830F2B1887820E6BF
:1004E000547FF5F0C39420500375F020E5F0B188F7
:1004F00008B830EBB1A1B1904002DAC5B1A122C079
:1005000083C082B1A19007F4D1F2D082D083C0839E
:10051000C082D104B1A14007B1A1D0E0D0E02290C7
:1005200008ABD1F2D082D083B1A122C082C0839027
:100530001238D1F2D083D082D1E5743AB188D1DCBF
:100540007428B188E0D183C082C08390089CD1F226
:10055000B1DE20D50C400AD083D082F0B1A1A3A196
:100560003890125FD1F2D083D082227A12B1A1EA00
:10057000C0E0F11BD0E0FAB1904002DAF2B1A12262
:100580003098FDC298E599223099FDF599C29922DB
:10059000C0E0C3309808E599B41B03D3C298D0E0FB
:1005A00022C0E0740DB188D0E022B180D1C3C3C2B3
:1005B000D5C2D2B40D03D2D522B41B02B322B400EB
:1005C00003D2D222B47F0280F8C0F0F5F0D1A5406A
:1005D00009C5F0B188C5F0D0F022D0F080CCB1AA26
:1005E00030D50122500122C4F5F0B1AA20D20F303B
:1005F000D506C2D5E5F0C42250012245F022740888
:10060000B18880DAC0E0E8C0E0E9C0E0EAC0E0EB31
:10061000C0E0B1AAF8405D20D55A20D2F5B1AAF9C0
:10062000405220D52B30D2067408B18880E4B1AA9C
:10063000FA404120D52130D2067408B18880DEB15D
:10064000AAFB403020D51A30D2207408B18880DE51
:100650007583008882801D758300E8C449F5828017
:10066000138883E9C44AF582800AE8C449F583EA1D
:10067000C44BF582D0E0FBD0E0FAD0E0F9D0E0F84E
:10068000D0E022C0E0C4D18DD0E0D18D22540F241F
:100690000383B1882230313233343536373839412B
:1006A0004243444546C3C0F09430F5F0940A4006F6
:1006B000E5F09407F5F0E5F0C354F06001D3E5F000
:1006C000D0F022C0F0F5F0C39461400B941A5007AB
:1006D000C3E5F09420F5F0E5F0D0F022C0E07420FE
:1006E000B188D0E022C0E0E583D183E582D183D018
:1006F000E022C0E0E4932098156010A2E7547F3018
:1007000099FDF599C2994003A380E9D0E022C298EF
:10071000E599B41BDF740DB18880F0D1E5E493A3B3
:10072000FBC083C08290102893FAEB90113893FE9F
:1007300054FC0303FFEE5403D082D083FE14600FF9
:10074000C0E0E493A3FCD0E0146004E493A3FDF1C3
:1007500081C082C083900EFEF1A9EFF8D0E0D0F006
:10076000C0F0C0E0FEE5F0FFE814C33375F07AC0D6
:10077000F075F007C0F09008BF73D083D082B1A1AC
:1007800022743AB188D1DCEBD183D1DCBE0104798B
:100790000B8011ECD183D1DCBE020479088005ED19
:1007A000D1837906D1DCD9FC227808EA930A18A211
:1007B000E7547FB188400280F2D1DCD8FC223E4C65
:1007C0006F633D003A202856657273696F6E203161
:1007D0002E302920436F6D6D616E643E004C6F6357
:1007E0006174696F6E2028003D44656661756C74A4
:1007F000293A20004E6577206D656D6F7279207003
:100800006F696E746572206C6F636174696F6E3AA4
:1008100020000D533D53696E676C652053746570FD
:100820002C204E3D4E6F726D616C202864656661B0
:10083000756C74292C203F3D48656C70203E00503B
:100840007265737320616E79206B65793A20000DB3
:100850000D52756E2066726F6D206D656D6F7279C9
:10086000206C6F616374696F6E2028000D0D496EF6
:1008700074657272757074207072696F72697479C0
:100880003E204C3D4C6F772C20483D4869676820DE
:100890002864656661756C74293A20002920204E11
:1008A00065772056616C75653A20002020436F6D96
:1008B0006D616E642041626F72746564210D002168
:1008C000A521B721BC21C121C621D121D821DE21FA
:1008D000E521F121FC4108410C4110411341164131
:1008E00019411C411F4127412E41324135413841B8
:1008F0003C413F4199414B41524159415D41644125
:1009000073417A41814188418C419341A241B04178
:10091000C341CA41D27452120588EB540712068DA6
:100920002274401205887452120588EB5401120695
:100930008D22EC20E705EC12068322900FBBE49396
:10094000A360F3F8C39C70041206F222E493A33070
:10095000E7FA80EAEC547823C4F8EC5480601590F0
:100960001128E893900F943582F582500205831286
:1009700006F28006E82420120683742E120588EC05
:10098000540712068D22EC20E708C33FFF500D0EDE
:10099000800AF404FCEFC39CFF50011EEE12068394
:1009A000EF12068322EE54F8F8EBC4035407481202
:1009B0000683EC1206832251F431152251F43132B0
:1009C0002251F431212251E851D951E2EC1206832F
:1009D00022313251D951E8223132EDFC21C851EE99
:1009E00051D931542251EE51D9742F120588315406
:1009F0002251F4313251D9EDFC31862251E851D9DE
:100A000051E2EC12068321F5311521FE312121FE40
:100A100051E82251EE223154223132223121225129
:100A2000E8744212058822311551D93186223132BB
:100A300021F531152251F922315421F53186225107
:100A4000D351E8742B12058851F922311551D9512F
:100A5000E822311551D9313222311521C8313251B4
:100A6000D9311522ECC0E0EDFC313251D9D0E0FC97
:100A7000313222313251D9312122312151D951E83B
:100A800022312151D9313222312121C8315451D959
:100A900051EE2251F951D951E2EC120683ED1206C2
:100AA000832251F451D351E8742B12058851F92255
:100AB00051F451D351E8742B1205887450120588F3
:100AC00051EE2251F451D351F92251D351F951D958
:100AD00051E822744012058822742C1205881206EF
:100AE000DC22742312058822744112058822744383
:100AF0001205882251E851D922C083C08290148700
:100B00001206F2D082D08322758130C2D3C2D412B1
:100B100002E9D299C29878081205A1D8FE900BD8A4
:100B20001206F2902000C082C0839007BE1206F227
:100B3000D083D0821206E5C082C0839007C412061B
:100B4000F21205801206C3F52090148CE493604BDA
:100B5000B52040A3E493C0E0A3E493D0F0C082C0EA
:100B600083F58285F0831206F21205A1D083D0822C
:100B7000A3E493F522E4A393F521D023D024900B92
:100B800026C082C083852482852383C021C022227F
:100B9000020B26A3A3A3A3A3020B4CD083D08212E3
:100BA00005A1020B26E9C0E0EAC0E0EBC0E0ECC022
:100BB000E0EDC0E0EEC0E0EFC0E086831886821270
:100BC000071BD0E0FFD0E0FED0E0FDD0E0FCD0E09D
:100BD000FBD0E0FAD0E0F9220D2020200D202020CB
:100BE00020202020200C57656C636F6D6520746F8A
:100BF00020746865206E657720616E6420706F7365
:100C00007369626C79206576656E20696D70726FAC
:100C10007665642038303331206D6F6E69746F7281
:100C20002F64656275676765720D62792050617522
:100C30006C2053746F6666726567656E206F6E20F8
:100C400031342D4F43542D393120666F72206E6F31
:100C500020676F6F6420726561736F6E20776861C3
:100C600074736F657665722E2E2E0D0D5468657344
:100C7000652061726520736F6D65206F66207468F2
:100C800065206665617475726573206F666665724E
:100C90006564206279207468697320706172746978
:100CA00063756C61722064656275676765723A0D81
:100CB0000D2020202020446F776E6C6F61642070BF
:100CC000726F6772616D732066726F6D2050432082
:100CD000202020202020202020557365722D467270
:100CE00069656E646C696E65737321212121210D24
:100CF000202020202052756E2050726F6772616D27
:100D000020202020202020202020202020202020E3
:100D1000202020202020202055736573206E6F2016
:100D200065787465726E616C2052414D0D202020F3
:100D300020202020284E6F726D616C2C206F722055
:100D400073696E676C652D7374657029202020208F
:100D500020202020203C4553433E206B65792069AC
:100D60007320737570706F727465640D202020207D
:100D7000204C69737420617373656D626C652063C8
:100D80006F64652066726F6D206D656D6F7279207E
:100D9000202020206175746F6D6174696320626129
:100DA0007564207261746520646574656374696F2D
:100DB0006E0D20202020204865782044756D70201D
:100DC000616E6420456469742065787465726E6133
:100DD0006C2052414D20202020204F6E2D6C696EDA
:100DE000652068656C7020287479706520273F271E
:100DF000290D0D486F77657665722C20796F752007
:100E0000646F6E27742067657420736F6D657468F6
:100E1000696E2720666F72206E6F7468696E272E68
:100E20002E2E202054686520636F646520666F72E3
:100E300020746869732064656275676765720D72F6
:100E400065717569726573207175697465206120BB
:100E5000626974206D6F726520726F6F6D207468A7
:100E6000616E206973207479706963616C20666FAC
:100E70007220612064656275676765722C206275F7
:100E8000742069742077696C6C20616C6C0D6669E4
:100E90007420696E746F2061203237363420283810
:100EA0004B2078203829204550524F4D2E0D0D4EA5
:100EB0004F20436F70797269676874212120205038
:100EC0006C656173652064697374726962757465B9
:100ED00020667265656C792E20204D616B652061FE
:100EE00073206D616E7920636F7069657320617323
:100EF00020796F752077616E742E0D0D0D004143C2
:100F0000414CCC004144C420414444C3414A4DD0EB
:100F1000414ECC434A4EC5434CD24350CC44C144CD
:100F200045C34449D6444A4EDA494EC34AC24A42AE
:100F3000C34AC34A4DD04A4EC24A4EC34A4EDA4A09
:100F4000DA4C43414CCC4C4A4DD04D4FD64D4F56C8
:100F5000C34D4F56D84D55CC4E4FD04F52CC504F1D
:100F6000D0505553C85245D4524554C952CC524C16
:100F7000C352D25252C3534554C2534A4DD0535513
:100F800042C2535741D05843C8584348C45852CC22
:100F90003F3FBF0050B054434FCE50B153434FCEAC
:100FA00050B249C550B349D043B05432434FCE50EC
:100FB00053D744B84143C3FDC2FE00E04143C3815F
:100FC00053D0824450CC834450C88050B09050B12C
:100FD000A050B2B050B399534255C6CD5448B2C890
:100FE0005432434FCECC544CB2CB5243415032C812
:100FF000CA5243415032CC8C5448B08A544CB08DC4
:101000005448B18B544CB1F0C2D05053D7A849C505
:10101000B849D089544D4FC48854434FCE98534358
:101020004FCE8750434FCE005A0E48732B2B2B2B9D
:101030002B2B2B2B2B2B2B2B3000437521212121EC
:1010400021212121212121212E0E676E060606066F
:10105000060606060606060638006A700A0A0A0A26
:101060000A0A0A0A0A0A0A0A330E5D5D5D5D5D5DC1
:101070005D5D5D5D5D5D5D5D3B00121212121212E1
:101080001212121212121212410E8F8F8F8F8F8F27
:101090008F8F8F8F8F8F8F8F3E005D354C4C4C4CD8
:1010A0004C4C4C4C4C4C4C4C7C0E124F244C4C4CED
:1010B0004C4C4C4C4C4C4C4C4C004C4F80808080E9
:1010C00080808080808080805D0E4C2B57924C4CBD
:1010D0004C4C4C4C4C4C4C4C12001C1C1515151512
:1010E0001515151515151515630E19198488888899
:1010F0008888888888888888600078781F278B8B04
:101100002727272727272727530E5353194C4C4CA3
:101110004C4C4C4C4C4C4C4C530053531C4C4C4C76
:101120004C4C4C4C4C4C4C4C000206080C0E101213
:1011300014161B1E20232425AD066F393946494954
:10114000595959595959595963066F3939464949B5
:1011500059595959595959596306AD39160E111132
:1011600009090909090909096306AD39160E1111A2
:10117000090909090909090966061A1F160E11113C
:10118000090909090909090966061A1F160E11112C
:10119000090909090909090966061A1F160E11111C
:1011A000090909090909090966062269161F9286B3
:1011B0007A7A7A7A7A7A7A7A660622A14D83868654
:1011C0007E7E7E7E7E7E7E7E9B06969D160E111115
:1011D00009090909090909092606225D4DAD8E8E06
:1011E00076767676767676762606423D2F2B3737DC
:1011F00033333333333333334606423D390E111123
:1012000009090909090909094606423D3957111119
:101210005252525252525252A5061111390E111108
:101220000909090909090909A9068989391A898950
:1012300071717171717171710D45646974696E6755
:101240002045787465726E616C2052414D2E2E2EB1
:101250003C4553433E20746F20717569740D002026
:101260002045646974696E672066696E6973686594
:10127000642C2074686973206C6F636174696F6E8D
:1012800020756E6368616E6765640D0D000D0D421B
:101290006567696E206173636969207472616E733A
:1012A0006D697373696F6E206F6620496E74656C2B
:1012B0002048455820666F726D61742066696C65C0
:1012C0002C206F72203C4553433E20746F20616296
:1012D0006F72740D0D00446F776E6C6F61642061E6
:1012E000626F7274656420627920757365720D0D8A
:1012F000000D0D0D0D446F776E6C6F616420636F90
:101300006D706C657465640D0D0052756E206E6FA6
:10131000726D616C6C79000D0C4E6F772072756E7A
:101320006E696E67207468652070726F6772616D98
:101330002E2E2E0D0D0052756E20696E2073696E73
:10134000676C652073746570206D6F6465000D0DAA
:101350005468652073696E676C65207374657020CE
:1013600072756E20666561747572652077696C6C44
:10137000206E6F742066756E6374696F6E20756E73
:101380006C65737320494E5431202870696E202398
:101390003133292069730D636F6E6E656374656404
:1013A00020746F2067726F756E64206F72206F7487
:1013B000686572776973652068656C64206C6F7707
:1013C0002E0D0D000D0C4E6F772072756E6E696ECE
:1013D0006720696E2073696E676C65207374657031
:1013E000206D6F64653A20203C5245543E3D646553
:1013F0006661756C742C203F3D48656C700D0D0066
:10140000536B697070696E67202D2D2D2D2D2D3E2B
:10141000004E6578742077696C6C206265202D2DF4
:101420003E000D4C6F633A2020496E7465726E6108
:101430006C2052616D204D656D6F727920436F6E27
:1014400074656E74730D004E65772041636320569A
:10145000616C75653A20000D517569742073696E71
:10146000676C652073746570206D6F64652C206EE9
:101470006F772072756E6E696E67206E6F726D6128
:101480006C6C792E0D0D0044505452003F1505032D
:10149000615214B003A444150E029B4E14BD04FF08
:1014A0004814D204BD4C14F1056B451528052B00DA
:1014B0002052756E2070726F6772616D00204E65EC
:1014C00077206D656D6F7279206C6F636174696FE1
:1014D0006E00204845582044756D70204D656D6F35
:1014E000727920746F207468652053637265656E2D
:1014F00000204C69737420617373656D626C792090
:10150000636F6465002048656C703F3F3F00204476
:101510006F776E6C6F61642070726F6772616D209F
:1015200066726F6D205043002045646974206578B1
:101530007465726E616C2072616D000C5468657325
:101540006520636F6D6D616E6473206172652063E9
:10155000757272656E746C7920737570706F7274C9
:1015600065643A0D0D000D416C6C206E756D6572F1
:101570006963616C2076616C7565732061726520AA
:1015800073686F776E20696E206865782E20205012
:1015900072657373696E67203C4553433E206B65EB
:1015A000792077696C6C2065786974207468650DA2
:1015B00063757272656E7420636F6D6D616E642CFD
:1015C000206576656E207768696C65206C69737438
:1015D000696E672F64756D70696E672E20204D6F80
:1015E00073742070726F6D70747320726571756999
:1015F000726520610D73696E676C65206368617246
:1016000061637465722C207479706963616C6C79A4
:1016100020746865206669727374206C65747465E3
:1016200072206F66207468652064657369726564F2
:10163000206F7074696F6E2E0D0D466F7220696E8B
:10164000666F726D6174696F6E2072656761726436
:10165000696E67207468652073696E676C652D73A9
:101660007465702072756E20666561747572652C84
:101670000D7479706520273F27207768656E20619B
:10168000736B6564202753696E676C652D73746591
:10169000702F4E6F726D616C27206265666F726588
:1016A0002072756E6E696E67207468652070726F47
:1016B0006772616D2E0D0D000C5468652073696EA4
:1016C000676C6520737465702072756E2066656145
:1016D0007475726520616C6C6F777320796F7520FB
:1016E000746F206578656375746520796F757220F5
:1016F00070726F6772616D2066726F6D206D656DBF
:101700006F72790D6F6E6520696E73747275637494
:10171000696F6E20617420612074696D652C20777B
:1017200068696C65206D6F6E69746F72696E672091
:101730007468652072656769737465727320616E81
:101740006420696E737472756374696F6E732E0DA5
:101750004974206974204E4F5420612073696D755F
:101760006C6174696F6E2C207468652070726F678D
:1017700072616D2069732065786563757465642096
:1017800062792074686520383033312F353120700C
:10179000726F636573736F722E0D45787465726E28
:1017A000616C20496E7465727275707420233120EB
:1017B0006D7573742062652068656C64206C6F774A
:1017C00020746F206D616B65207468652073696E8D
:1017D000676C6520737465702066756E6374696FDD
:1017E0006E2E0D0D446573706974652061747465A7
:1017F0006D70747320746F206D616B652074686503
:101800002073696E676C6520737465702072756EE5
:1018100020636F6D70617469626C652077697468AC
:1018200020616C6C2070726F6772616D732C0D7427
:10183000686572652077696C6C20616C776179737B
:1018400020626520736F6D65206261736963206C2F
:10185000696D69746174696F6E7320647565207455
:101860006F20697473206E61747572653A0D0D2076
:10187000312D2045787465726E616C20496E7465F7
:101880007272757074202331206D757374206E6FC1
:10189000742062652064697361626C65642C2065E4
:1018A0002E672E204D4F562049452C233831680D88
:1018B00020322D2054696D6572202331206D75739F
:1018C0007420626520636F72726563746C7920673F
:1018D000656E65726174696E672020746865206248
:1018E000617564207261746520666F72207468652A
:1018F0002073657269616C20706F72740D20332DD6
:1019000020544920616E642052492077696C6C2014
:101910006E6F7420776F726B206E6F726D616C6C7E
:10192000792C20652E672E20323030333A204A4EF3
:10193000422052492C323030332C2075736520738D
:101940006B69702E2E2E0D20342D20496E74657219
:1019500072757074732077696C6C206E6F74206779
:1019600065742073657276696365206F722077698C
:101970006C6C20696E746572727570742074686521
:101980002073696E676C6520737465700D20352D4A
:101990002041626F75742033302062797465732042
:1019A0006F66207370616365206D75737420626566
:1019B000206C65667420617661696C61626C65207B
:1019C0006F6E2074686520737461636B210D20361F
:1019D0002D203F3F3F20204F746865722070726F4A
:1019E000626C656D73206D617920616C736F206529
:1019F000786973742C2028746869732070726F671B
:101A000072616D20697320465245452C20796F75AF
:101A1000206B6E6F77290D0D5065726861707320B1
:101A200074686520776F727374206C696D69746176
:101A300074696F6E206F66207468652073696E67C5
:101A40006C6520737465702072756E2069732074E4
:101A50006861742069742074616B657320610D7610
:101A6000657279206C6F6E672074696D6520746F84
:101A70002065786563757465206576656E2073688A
:101A80006F727420706965636573206F6620636F81
:101A900064652E20204974206973207265636F6D20
:101AA0006D656E64656420746861740D61206E6F8D
:101AB000726D616C2072756E206265206174746550
:101AC0006D7074656420666972737420746F20652C
:101AD0007374696D617465207768657265207468D8
:101AE000652070726F6772616D20676F657320612A
:101AF00073747261792C0D74686520617474656DFE
:101B0000707420612073696E676C652073746570F2
:101B10002061742074686520626567696E6E696E05
:101B200067206F6620746865207175657374696FCE
:101B30006E61626C6520636F64652C2077697468E0
:101B400020610D68617264636F7079206F66207424
:101B5000686520617373656D626C79206C6973745C
:101B6000696E672066696C65206F6E2D68616E64B2
:101B700020666F72206D656D6F7279206C6F636186
:101B800074696F6E207265666572656E63652E0D91
:101B90000D000C4265747765656E20737465707313
:101BA0002C20746865206D6F6E69746F7220757378
:101BB0006573206162736F6C7574656C79204E4F2C
:101BC00020696E7465726E616C206F722065787426
:101BD00065726E616C206D656D6F72792E0D486F48
:101BE00077657665722C2061626F757420333020C2
:101BF0006279746573206F6620737461636B207300
:101C000070616365206D757374206265206C656614
:101C10007420617661696C61626C652E2E2E0D0DEB
:101C2000447572696E6720612073696E676C652008
:101C3000737465702072756E2C2070726573736991
:101C40006E672052455455524E207265706561741E
:101C500065646C792077696C6C20626520746865B6
:101C600020757375616C20636F757273650D6F6697
:101C700020616374696F6E2E2020486F77657665EA
:101C8000722C206F74686572206F7074696F6E7348
:101C90002061726520617661696C61626C652E0DF0
:101CA0000D2020202020202020202020205479706A
:101CB000696E6720273F272077696C6C2064697301
:101CC000706C617920746869732068656C7020732A
:101CD000637265656E0D0D0053696E676C65205308
:101CE00074657020436F6D6D616E64733A0D0D20E5
:101CF0003C5245543E202020205072696E7420537F
:101D0000746174757320616E6420657865637574A1
:101D10006520746865206E65787420696E737472CE
:101D2000756374696F6E0D203C53504143453E20EE
:101D30002045786563757465206E65787420696EDA
:101D4000737472756374696F6E20772F6F7574206A
:101D5000737461747573206C696E65730D20202730
:101D60003F272020202020446973706C6179207403
:101D7000686973206F6E2D6C696E652068656C7084
:101D80000D202027522720202020205072696E74B9
:101D9000206F7574205370656369616C2046756EA1
:101DA0006374696F6E205265676973746572730D31
:101DB000202027482720202020204865782064758F
:101DC0006D7020696E7465726E616C2072616D0D4C
:101DD00020202753272020202020536B6970207457
:101DE00068697320696E737472756374696F6E0DC0
:101DF000202027412720202020204368616E67652E
:101E00002074686520416363756D756C61746F72D1
:101E100027732076616C75650D20202751272020BF
:101E2000202020517569742053696E676C652053BA
:101E30007465702C20636F6E74696E7565206578AB
:101E400065637574696E67206E6F726D616C6C7915
:031E50000D0D0075
:00000001FF
